BL51 BANKED LINKER/LOCATER V6.22.2.0                                                    03/16/2023  09:24:19  PAGE 1


BL51 BANKED LINKER/LOCATER V6.22.2.0, INVOKED BY:
C:\KEIL_V5\C51\BIN\BL51.EXE .\Release\system_FE81001.obj, .\Release\main.obj TO .\Release\Sample_DrvGPIO REGFILE (.\Rele
>> ase\Sample_DrvGPIO.ORC) PRINT (.\Sample_DrvGPIO.m51) RAMSIZE (256) CODE (0X0000-0X1FFF) XDATA (0X8000-0X87FF)


MEMORY MODEL: SMALL


INPUT MODULES INCLUDED:
  .\Release\system_FE81001.obj (SYSTEM_FE81001)
  .\Release\main.obj (MAIN)
  C:\KEIL_V5\C51\LIB\C51S.LIB (?C_STARTUP)


LINK MAP OF MODULE:  .\Release\Sample_DrvGPIO (SYSTEM_FE81001)


            TYPE    BASE      LENGTH    RELOCATION   SEGMENT NAME
            -----------------------------------------------------

            * * * * * * *   D A T A   M E M O R Y   * * * * * * *
            REG     0000H     0008H     ABSOLUTE     "REG BANK 0"
            DATA    0008H     0006H     UNIT         ?DT?_DELAY?MAIN
            IDATA   000EH     0001H     UNIT         ?STACK

            * * * * * * *   C O D E   M E M O R Y   * * * * * * *
            CODE    0000H     0003H     ABSOLUTE     
            CODE    0003H     0043H     UNIT         ?PR?IOCONFIG?MAIN
            CODE    0046H     003DH     UNIT         ?PR?MAIN?MAIN
            CODE    0083H     003BH     UNIT         ?PR?_DELAY?MAIN
            CODE    00BEH     000CH     UNIT         ?PR?CLOCK_CONFIG?MAIN
            CODE    00CAH     000CH     UNIT         ?C_C51STARTUP
            CODE    00D6H     0001H     UNIT         ?PR?SYSTEMINIT?SYSTEM_FE81001



OVERLAY MAP OF MODULE:   .\Release\Sample_DrvGPIO (SYSTEM_FE81001)


SEGMENT
  +--> CALLED SEGMENT
---------------------
?C_C51STARTUP
  +--> ?PR?MAIN?MAIN

?PR?MAIN?MAIN
  +--> ?PR?CLOCK_CONFIG?MAIN
  +--> ?PR?IOCONFIG?MAIN



SYMBOL TABLE OF MODULE:  .\Release\Sample_DrvGPIO (SYSTEM_FE81001)

  VALUE           TYPE          NAME
  ----------------------------------

  -------         MODULE        SYSTEM_FE81001
  C:0000H         SYMBOL        _ICE_DUMMY_
BL51 BANKED LINKER/LOCATER V6.22.2.0                                                  03/16/2023  09:24:19  PAGE 2


  C:00D6H         PUBLIC        SystemInit
  -------         PROC          SYSTEMINIT
  C:00D6H         LINE#         38
  C:00D6H         LINE#         39
  C:00D6H         LINE#         41
  -------         ENDPROC       SYSTEMINIT
  -------         ENDMOD        SYSTEM_FE81001

  -------         MODULE        MAIN
  C:0000H         SYMBOL        _ICE_DUMMY_
  D:0090H         PUBLIC        P1
  D:00B0H         PUBLIC        P3
  D:00A8H         PUBLIC        IE
  C:0083H         PUBLIC        _delay
  D:00B8H         PUBLIC        IP
  C:0046H         PUBLIC        main
  C:00BEH         PUBLIC        Clock_Config
  D:0098H         PUBLIC        SCON
  D:0088H         PUBLIC        TCON
  D:00C8H         PUBLIC        T2CON
  C:0003H         PUBLIC        IOConfig
  D:00D0H         PUBLIC        PSW
  -------         PROC          _DELAY
  D:0008H         SYMBOL        cnt
  -------         DO            
  D:000AH         SYMBOL        i
  D:000CH         SYMBOL        j
  -------         ENDDO         
  C:0083H         LINE#         31
  C:0087H         LINE#         32
  C:0087H         LINE#         35
  C:0098H         LINE#         36
  C:00BDH         LINE#         38
  -------         ENDPROC       _DELAY
  -------         PROC          CLOCK_CONFIG
  C:00BEH         LINE#         50
  C:00BEH         LINE#         51
  C:00BEH         LINE#         52
  C:00C9H         LINE#         53
  -------         ENDPROC       CLOCK_CONFIG
  -------         PROC          IOCONFIG
  C:0003H         LINE#         56
  C:0003H         LINE#         57
  C:0003H         LINE#         59
  C:0024H         LINE#         62
  C:0045H         LINE#         63
  -------         ENDPROC       IOCONFIG
  -------         PROC          MAIN
  C:0046H         LINE#         75
  C:0046H         LINE#         76
  C:0046H         LINE#         77
  C:0049H         LINE#         78
  C:004CH         LINE#         80
  C:0051H         LINE#         81
  C:0057H         LINE#         82
  C:005CH         LINE#         85
  C:005CH         LINE#         86
BL51 BANKED LINKER/LOCATER V6.22.2.0                                                  03/16/2023  09:24:19  PAGE 3


  C:005CH         LINE#         87
  C:0073H         LINE#         88
  C:0073H         LINE#         89
  C:0078H         LINE#         90
  C:007AH         LINE#         92
  C:007AH         LINE#         93
  C:0080H         LINE#         94
  C:0080H         LINE#         95
  -------         ENDPROC       MAIN
  -------         ENDMOD        MAIN



FUNCTION REGISTER MASKS


FUNCTION . . . . REG MASK
-------------------------

CLOCK_CONFIG . . @0xe301
IOCONFIG . . . . @0xe301
MAIN . . . . . . @0xf303
SYSTEMINIT . . . @0x8000
_DELAY . . . . . @0xf000

*** WARNING L16: UNCALLED SEGMENT, IGNORED FOR OVERLAY PROCESS
    SEGMENT: ?PR?SYSTEMINIT?SYSTEM_FE81001

*** WARNING L16: UNCALLED SEGMENT, IGNORED FOR OVERLAY PROCESS
    SEGMENT: ?PR?_DELAY?MAIN

Program Size: data=15.0 xdata=0 code=215
LINK/LOCATE RUN COMPLETE.  2 WARNING(S),  0 ERROR(S)
